:100000000C9434000C9451000C9451000C94510049
:100010000C9451000C9451000C9451000C94E50088
:100020000C9451000C9451000C9451000C94B400A9
:100030000C9451000C9451000C9483000C945100CA
:100040000C9451000C9451000C9451000C945100EC
:100050000C9451000C9451000C9451000C945100DC
:100060000C9451000C94510011241FBECFEFD8E026
:10007000DEBFCDBF11E0A0E0B1E0EAEAF5E002C0EA
:1000800005900D92A031B107D9F721E0A0E1B1E0D0
:1000900001C01D92A531B207E1F70E9433010C9413
:1000A000D3020C9400008230910561F083309105F9
:1000B00099F00197C9F416BC80916E00826080931C
:1000C0006E0016C0109285001092840080916F001F
:1000D000826080936F000CC01092B200809170001B
:1000E00082608093700004C081E090E00E94D3029F
:1000F00078949FB7F894809112019FBF8823C9F329
:100100001092120108951F920F920FB60F921124B0
:100110002F933F938F939F938091100190911101A2
:10012000019690931101809310018091120181300A
:1001300091F0209110013091110180911301909163
:1001400014012817390738F081E0809312011092CA
:100150001101109210019F918F913F912F910F905B
:100160000FBE0F901F9018951F920F920FB60F920F
:1001700011242F933F938F939F938091100190911F
:100180001101019690931101809310018091120149
:10019000813091F020911001309111018091130173
:1001A000909114012817390738F081E080931201EB
:1001B00010921101109210019F918F913F912F91F8
:1001C0000F900FBE0F901F9018951F920F920FB6B1
:1001D0000F9211242F933F938F939F93809110013F
:1001E00090911101019690931101809310018091DB
:1001F0001201813091F02091100130911101809114
:100200001301909114012817390738F081E0809389
:10021000120110921101109210019F918F913F9144
:100220002F910F900FBE0F901F901895FC01219AEF
:1002300085E290E09387828785B5836085BD21E064
:1002400030E03587248782E090E09093140180931A
:10025000130184B5826084BD89EF87BD3787268707
:1002600080E090E00895CF92DF92EF92FF9280E0DD
:1002700091E00E941601C12CD12C760160E070E063
:10028000CB01609300017093010180930201909370
:10029000030180910E0190910F010E945300E091A3
:1002A0000A01F0910B018081826080838FEFC81A70
:1002B000D80AE80AF80AC701B6010E94D8012FE659
:1002C00032E143E05BE30E94660220E030E0A901F6
:1002D0000E946C01D6CF5058BB27AA270E948301E9
:1002E0000C942C020E941E0238F00E94250220F07D
:1002F00039F49F3F19F426F40C941B020EF4E09598
:10030000E7FB0C941502E92F0E943D0258F3BA173F
:10031000620773078407950720F079F4A6F50C941B
:100320005F020EF4E0950B2EBA2FA02D0B01B90140
:1003300090010C01CA01A0011124FF27591B99F05B
:10034000593F50F4503E68F11A16F040A22F232F67
:10035000342F4427585FF3CF469537952795A795B7
:10036000F0405395C9F77EF41F16BA0B620B730B5E
:10037000840BBAF09150A1F0FF0FBB1F661F771FCF
:10038000881FC2F70EC0BA0F621F731F841F48F484
:10039000879577956795B795F7959E3F08F0B0CF0D
:1003A0009395880F08F09927EE0F979587950895F4
:1003B000E89409C097FB3EF49095809570956195FF
:1003C0007F4F8F4F9F4F9923A9F0F92F96E9BB27B5
:1003D0009395F695879577956795B795F111F8CF31
:1003E000FAF4BB0F11F460FF1BC06F5F7F4F8F4F9C
:1003F0009F4F16C0882311F096E911C0772321F092
:100400009EE8872F762F05C0662371F096E8862F29
:1004100070E060E02AF09A95660F771F881FDAF780
:10042000880F9695879597F9089597F99F6780E8C3
:1004300070E060E008959FEF80EC089500240A9436
:100440001616170618060906089500240A941216AF
:100450001306140605060895092E0394000C11F4E2
:10046000882352F0BB0F40F4BF2B11F460FF04C08F
:100470006F5F7F4F8F4F9F4F089557FD9058440FE8
:10048000551F59F05F3F71F04795880F97FB991FF3
:1004900061F09F3F79F087950895121613061406B0
:1004A000551FF2CF4695F1DF08C01616170618063D
:1004B000991FF1CF86957105610508940895E89418
:1004C000BB2766277727CB0197F908950E94790209
:1004D0000C942C020E941E0238F00E94250220F08B
:1004E000952311F00C9415020C941B0211240C940A
:1004F00060020E943D0270F3959FC1F3950F50E09A
:10050000551F629FF001729FBB27F00DB11D639FC5
:10051000AA27F00DB11DAA1F649F6627B00DA11D6B
:10052000661F829F2227B00DA11D621F739FB00D11
:10053000A11D621F839FA00D611D221F749F332781
:10054000A00D611D231F849F600D211D822F762F1A
:100550006A2F11249F5750409AF0F1F088234AF0F7
:10056000EE0FFF1FBB1F661F771F881F9150504063
:10057000A9F79E3F510580F00C9415020C9460027F
:100580005F3FE4F3983ED4F3869577956795B795EA
:10059000F795E7959F5FC1F7FE2B880F911D969504
:0A05A000879597F90895F894FFCFAE
:1005AA000000000000006F12033B00000000000082
:00000001FF
